:100000000C9472000C948D000C948D000C948D0057
:100010000C948D000C948D000C948D000C948D002C
:100020000C948D000C948D000C948D000C948D001C
:100030000C948D000C948D000C948D000C948D000C
:100040000C948D000C948D000C948D000C948D00FC
:100050000C948D000C948D000C948D000C948D00EC
:100060000C948D000C948D000C948D000C948D00DC
:100070000C948D000C948D000C948D000C948D00CC
:100080000C948D000C948D000C948D000C948D00BC
:100090000C948D000C948D000C948D000C948D00AC
:1000A0000C948D000C948D000C948D000C948D009C
:1000B0000C948D000C948D000C948D000C948D008C
:1000C0000C948D000C948D000C948D000C948D007C
:1000D0000C948D000C948D000C948D000C948D006C
:1000E0000C948D0011241FBECFEFD1E2DEBFCDBF37
:1000F00000E00CBF84B78093000214BE0FB6F894E2
:10010000A8958091600088618093600010926000E3
:100110000FBE0E94A1000C94BE000C940000E8E009
:10012000F1E080818E7F808381B38F5F81BB80818E
:100130008160808385E08A95F1F7000090E080E09F
:100140000895F8948FEF80BB8091070181608093C0
:10015000070111BA809108018160809308017894A9
:1001600088E19EE00FB6F894A895809360000FBEDA
:1001700090936000A8950E948F00FCCFF894FFCF69
:00000001FF
